 srvkm

 Timestamp is 4beb96ec (Thu May 13 15:06:36 2010)

 Preferred load address is 10000000

 Start         Length     Name                   Class
 0001:00000000 00000004H .CRT$XCA                CODE
 0001:00000004 00000004H .CRT$XCZ                CODE
 0001:00000008 00000004H .CRT$XIA                CODE
 0001:0000000c 00000004H .CRT$XIZ                CODE
 0001:00000010 00000004H .CRT$XPA                CODE
 0001:00000014 00000004H .CRT$XPZ                CODE
 0001:00000018 00000004H .CRT$XTA                CODE
 0001:0000001c 00000004H .CRT$XTZ                CODE
 0001:00000020 00000dc6H .rdata                  CODE
 0001:00000de8 00000022H .rdata$debug            CODE
 0001:00000e0c 000147e0H .text                   CODE
 0001:000155ec 00000034H .xdata                  CODE
 0001:00015620 00000028H .idata$2                CODE
 0001:00015648 00000014H .idata$3                CODE
 0001:0001565c 000000fcH .idata$4                CODE
 0001:00015758 00000016H .idata$6                CODE
 0001:00015770 000000edH .edata                  CODE
 0002:00000000 000000fcH .idata$5                DATA
 0002:00000100 0000f208H .data                   DATA
 0002:0000f320 00000804H .bss                    DATA
 0003:00000000 00000e58H .pdata                  DATA

  Address         Publics by Value              Rva+Base       Lib:Object

 0000:00000000       ___safe_se_handler_count   00000000     <absolute>
 0000:00000000       ___safe_se_handler_table   00000000     <absolute>
 0001:00000000       __xc_a                     10001000     corelib0:crt0init.obj
 0001:00000004       __xc_z                     10001004     corelib0:crt0init.obj
 0001:00000008       __xi_a                     10001008     corelib0:crt0init.obj
 0001:0000000c       __xi_z                     1000100c     corelib0:crt0init.obj
 0001:00000010       __xp_a                     10001010     corelib0:crt0init.obj
 0001:00000014       __xp_z                     10001014     corelib0:crt0init.obj
 0001:00000018       __xt_a                     10001018     corelib0:crt0init.obj
 0001:0000001c       __xt_z                     1000101c     corelib0:crt0init.obj
 0001:00000040       ??_C@_1FE@MFCHHLJM@?$AAk?$AAe?$AAr?$AAn?$AAe?$AAl?$AA?5?$AAI?$AAO?$AAC?$AAT?$AAL?$AA_?$AAP?$AAO?$AAW?$AAE?$AAR?$AA_?$AAS?$AAE?$AAT?$AA?5?$AAs?$AAe?$AAt?$AAt?$AAi?$AAn?$AAg?$AA?5?$AAs@ 10001040     pvr_bridge_k.obj
 0001:00000094       ??_C@_15MAOEGKJF@?$AA?$CF?$AAS?$AA?$AA@ 10001094     osfunc_srvkm.obj
 0001:0000009c       ??_C@_0BG@OLGOIILN@PVRSRV_EVENTOBJECT_?$CFd?$AA@ 1000109c     osfunc_srvkm.obj
 0001:000000b4       ??_C@_1CC@HNHLKECD@?$AA?$CI?$AAe?$AAr?$AAr?$AAo?$AAr?$AA?5?$AAc?$AAo?$AAd?$AAe?$AA?3?$AA?5?$AA?$CF?$AAd?$AA?$CJ?$AA?$AA@ 100010b4     osfunc_srvkm.obj
 0001:000000d8       ??_C@_1ME@PMFLDMJM@?$AAH?$AA?3?$AA?2?$AAW?$AAI?$AAN?$AAC?$AAE?$AA6?$AA0?$AA0?$AA?2?$AAP?$AAL?$AAA?$AAT?$AAF?$AAO?$AAR?$AAM?$AA?2?$AAS?$AAM?$AAD?$AAK?$AAV?$AA2?$AA1?$AA0?$AA?2?$AAS?$AAR@ 100010d8     osfunc_srvkm.obj
 0001:0000019c       ??_C@_1CI@OHCJFJPM@?$AAE?$AAR?$AAR?$AAO?$AAR?$AA?3?$AA?5?$AA?$CF?$AAs?$AA?5?$AAl?$AAi?$AAn?$AAe?$AA?5?$AA?$CF?$AAd?$AA?3?$AA?5?$AA?$AA@ 1000119c     osfunc_srvkm.obj
 0001:000001c4       ??_C@_1CK@MPGKAOE@?$AA?$CI?$AAe?$AAr?$AAr?$AAo?$AAr?$AA?5?$AAc?$AAo?$AAd?$AAe?$AA?3?$AA?5?$AA?$CF?$AAd?$AA?$CJ?$AA?3?$AA?5?$AA?$CF?$AAs?$AA?$AA@ 100011c4     osfunc_srvkm.obj
 0001:000001f0       ??_C@_09KBHAHJDF@?2PowerVR?2?$AA@ 100011f0     registry.obj
 0001:000001fc       ??_C@_01LFCBOECM@?4?$AA@   100011fc     srvkmcmn:pvrsrv.obj
 0001:00000200       ??_C@_03JALODAI@?$CFld?$AA@ 10001200     srvkmcmn:pvrsrv.obj
 0001:00000204       ??_C@_02NCJKDDL@?6?$AA?$AA@ 10001204     srvkmcmn:pvrsrv.obj
 0001:00000208       ??_C@_0CP@BIENFAHM@?6Application?5Context?5?$CIhDevMemCon@ 10001208     srvkmcmn:pvrsrv.obj
 0001:00000238       ??_C@_0BC@PNPFJMEC@?6Kernel?5Context?3?6?$AA@ 10001238     srvkmcmn:pvrsrv.obj
 0001:0000024c       ??_C@_0BD@FELDEKBN@?6?6Device?5Type?5?$CFd?3?6?$AA@ 1000124c     srvkmcmn:pvrsrv.obj
 0001:00000260       ??_C@_0BH@KCGJGLPH@?6Local?5Backing?5Store?3?6?$AA@ 10001260     srvkmcmn:pvrsrv.obj
 0001:00000278       ??_C@_0BK@CJAANPAB@PVRSRV_GLOBAL_EVENTOBJECT?$AA@ 10001278     srvkmcmn:pvrsrv.obj
 0001:00000294       ??_C@_04FOPLNFFP@span?$AA@ 10001294     srvkmcmn:ra.obj
 0001:0000029c       ??_C@_04LIAPHEDB@free?$AA@ 1000129c     srvkmcmn:ra.obj
 0001:000002a4       ??_C@_04GLMHKBCH@live?$AA@ 100012a4     srvkmcmn:ra.obj
 0001:000002ac       ??_C@_04HCPOGDOG@junk?$AA@ 100012ac     srvkmcmn:ra.obj
 0001:000002b4       ??_C@_0CH@PLGDNCLG@?7base?$DN0x?$CFx?5size?$DN0x?$CFx?5type?$DN?$CFs?5ref@ 100012b4     srvkmcmn:ra.obj
 0001:000002dc       ??_C@_0DF@OLDHKALG@?5?5error?3?5tail?5boundary?5tag?5has?5i@ 100012dc     srvkmcmn:ra.obj
 0001:00000314       ??_C@_0DF@LCJMIKHC@?5?5error?3?5head?5boundary?5tag?5has?5i@ 10001314     srvkmcmn:ra.obj
 0001:0000034c       ??_C@_0BC@EDPCNOOG@?5?5segment?5Chain?3?6?$AA@ 1000134c     srvkmcmn:ra.obj
 0001:00000360       ??_C@_0BD@MBBIMKGJ@export?5count?7?7?$CFlu?6?$AA@ 10001360     srvkmcmn:ra.obj
 0001:00000374       ??_C@_0BD@OLIIOHPB@import?5count?7?7?$CFlu?6?$AA@ 10001374     srvkmcmn:ra.obj
 0001:00000388       ??_C@_0BC@KNACCNA@total?5frees?7?7?$CFlu?6?$AA@ 10001388     srvkmcmn:ra.obj
 0001:0000039c       ??_C@_0BD@EOGCHLKO@total?5allocs?7?7?$CFlu?6?$AA@ 1000139c     srvkmcmn:ra.obj
 0001:000003b0       ??_C@_0CA@CINBBMOA@free?5resource?5count?7?$CFlu?5?$CI0x?$CFx?$CJ?6?$AA@ 100013b0     srvkmcmn:ra.obj
 0001:000003d0       ??_C@_0BI@LEJJMIMP@free?5segment?5count?7?$CFlu?6?$AA@ 100013d0     srvkmcmn:ra.obj
 0001:000003e8       ??_C@_0BI@FIAOCDCI@live?5segment?5count?7?$CFlu?6?$AA@ 100013e8     srvkmcmn:ra.obj
 0001:00000400       ??_C@_0BB@IDANMOJI@span?5count?7?7?$CFlu?6?$AA@ 10001400     srvkmcmn:ra.obj
 0001:00000414       ??_C@_0DD@BBMPLEDC@?5?5allocCB?$DN?$CF08X?5freeCB?$DN?$CF08X?5handl@ 10001414     srvkmcmn:ra.obj
 0001:00000448       ??_C@_0O@FCFOECN@?6Arena?5?8?$CFs?8?3?6?$AA@ 10001448     srvkmcmn:ra.obj
 0001:00000458       ??_C@_1M@NPGHCEML@?$AAP?$AAW?$AAC?$AA0?$AA?3?$AA?$AA@ 10001458     system:sysconfig.obj
 0001:00000464       ??_C@_0BD@ODPPLAIN@SGXGetClientInfoBW?$AA@ 10001464     srvkmbridged:bridged_sgx_bridge.obj
 0001:00000478       ??_C@_0CA@EIFFKNMN@PVRSRV_BRIDGE_SGX_GETCLIENTINFO?$AA@ 10001478     srvkmbridged:bridged_sgx_bridge.obj
 0001:00000498       ??_C@_0BH@OJNGMMEM@SGXReleaseClientInfoBW?$AA@ 10001498     srvkmbridged:bridged_sgx_bridge.obj
 0001:000004b0       ??_C@_0CE@HLNOPLNM@PVRSRV_BRIDGE_SGX_RELEASECLIENTI@ 100014b0     srvkmbridged:bridged_sgx_bridge.obj
 0001:000004d4       ??_C@_0BI@BLJIIEEG@SGXGetInternalDevInfoBW?$AA@ 100014d4     srvkmbridged:bridged_sgx_bridge.obj
 0001:000004ec       ??_C@_0CF@BIBINDHJ@PVRSRV_BRIDGE_SGX_GETINTERNALDEV@ 100014ec     srvkmbridged:bridged_sgx_bridge.obj
 0001:00000514       ??_C@_0M@MNGMALBD@SGXDoKickBW?$AA@ 10001514     srvkmbridged:bridged_sgx_bridge.obj
 0001:00000520       ??_C@_0BJ@NODNCHPG@PVRSRV_BRIDGE_SGX_DOKICK?$AA@ 10001520     srvkmbridged:bridged_sgx_bridge.obj
 0001:0000053c       ??_C@_0CC@KICAJGOF@PVRSRV_BRIDGE_SGX_GETPHYSPAGEADD@ 1000153c     srvkmbridged:bridged_sgx_bridge.obj
 0001:00000560       ??_C@_0CE@IIGLPIN@PVRSRV_BRIDGE_SGX_READREGISTRYDW@ 10001560     srvkmbridged:bridged_sgx_bridge.obj
 0001:00000584       ??_C@_0CC@BMPJGMNO@PVRSRV_BRIDGE_SGX_SCHEDULECOMMAN@ 10001584     srvkmbridged:bridged_sgx_bridge.obj
 0001:000005a8       ??_C@_0BK@ELJGOEFO@SGX2DQueryBlitsCompleteBW?$AA@ 100015a8     srvkmbridged:bridged_sgx_bridge.obj
 0001:000005c4       ??_C@_0CG@FICPHDGB@PVRSRV_BRIDGE_SGX_2DQUERYBLTSCOM@ 100015c4     srvkmbridged:bridged_sgx_bridge.obj
 0001:000005ec       ??_C@_07MMEBMBFO@DummyBW?$AA@ 100015ec     srvkmbridged:bridged_sgx_bridge.obj
 0001:000005f4       ??_C@_0BP@MOHANIJB@PVRSRV_BRIDGE_SGX_GETMMUPDADDR?$AA@ 100015f4     srvkmbridged:bridged_sgx_bridge.obj
 0001:00000614       ??_C@_0BE@GMHMJHCI@SGXSubmitTransferBW?$AA@ 10001614     srvkmbridged:bridged_sgx_bridge.obj
 0001:00000628       ??_C@_0CB@LGMDDJFH@PVRSRV_BRIDGE_SGX_SUBMITTRANSFER@ 10001628     srvkmbridged:bridged_sgx_bridge.obj
 0001:0000064c       ??_C@_0BB@BKDEILJN@SGXGetMiscInfoBW?$AA@ 1000164c     srvkmbridged:bridged_sgx_bridge.obj
 0001:00000660       ??_C@_0BO@LGACKMBI@PVRSRV_BRIDGE_SGX_GETMISCINFO?$AA@ 10001660     srvkmbridged:bridged_sgx_bridge.obj
 0001:00000680       ??_C@_0BH@MLEEJLHE@SGXGetInfoForSrvinitBW?$AA@ 10001680     srvkmbridged:bridged_sgx_bridge.obj
 0001:00000698       ??_C@_0CC@MKMFBNIA@PVRSRV_BRIDGE_SGXINFO_FOR_SRVINI@ 10001698     srvkmbridged:bridged_sgx_bridge.obj
 0001:000006bc       ??_C@_0BC@LDHGKCEG@SGXDevInitPart2BW?$AA@ 100016bc     srvkmbridged:bridged_sgx_bridge.obj
 0001:000006d0       ??_C@_0BP@FAAFBBEP@PVRSRV_BRIDGE_SGX_DEVINITPART2?$AA@ 100016d0     srvkmbridged:bridged_sgx_bridge.obj
 0001:000006f0       ??_C@_0BG@OKDAEDNB@SGXFindSharedPBDescBW?$AA@ 100016f0     srvkmbridged:bridged_sgx_bridge.obj
 0001:00000708       ??_C@_0CD@JIBIOMKF@PVRSRV_BRIDGE_SGX_FINDSHAREDPBDE@ 10001708     srvkmbridged:bridged_sgx_bridge.obj
 0001:0000072c       ??_C@_0BH@MIGJEHIE@SGXUnrefSharedPBDescBW?$AA@ 1000172c     srvkmbridged:bridged_sgx_bridge.obj
 0001:00000744       ??_C@_0CE@CCIPBGJL@PVRSRV_BRIDGE_SGX_UNREFSHAREDPBD@ 10001744     srvkmbridged:bridged_sgx_bridge.obj
 0001:00000768       ??_C@_0BF@GDJMNKNG@SGXAddSharedPBDescBW?$AA@ 10001768     srvkmbridged:bridged_sgx_bridge.obj
 0001:00000780       ??_C@_0CC@EJOCNPKJ@PVRSRV_BRIDGE_SGX_ADDSHAREDPBDES@ 10001780     srvkmbridged:bridged_sgx_bridge.obj
 0001:000007a4       ??_C@_0BN@PDPOCOPK@SGXRegisterHWRenderContextBW?$AA@ 100017a4     srvkmbridged:bridged_sgx_bridge.obj
 0001:000007c4       ??_C@_0CN@FLINDIJH@PVRSRV_BRIDGE_SGX_REGISTER_HW_RE@ 100017c4     srvkmbridged:bridged_sgx_bridge.obj
 0001:000007f4       ??_C@_0BJ@DCIOGPMF@SGXFlushHWRenderTargetBW?$AA@ 100017f4     srvkmbridged:bridged_sgx_bridge.obj
 0001:00000810       ??_C@_0CJ@CCNEDCPA@PVRSRV_BRIDGE_SGX_FLUSH_HW_RENDE@ 10001810     srvkmbridged:bridged_sgx_bridge.obj
 0001:0000083c       ??_C@_0BP@MPPABBB@SGXUnregisterHWRenderContextBW?$AA@ 1000183c     srvkmbridged:bridged_sgx_bridge.obj
 0001:0000085c       ??_C@_0CP@BFBHDDGD@PVRSRV_BRIDGE_SGX_UNREGISTER_HW_@ 1000185c     srvkmbridged:bridged_sgx_bridge.obj
 0001:0000088c       ??_C@_0BP@IDPLDJMB@SGXRegisterHWTransferContextBW?$AA@ 1000188c     srvkmbridged:bridged_sgx_bridge.obj
 0001:000008ac       ??_C@_0CP@BKGIBLMC@PVRSRV_BRIDGE_SGX_REGISTER_HW_TR@ 100018ac     srvkmbridged:bridged_sgx_bridge.obj
 0001:000008dc       ??_C@_0CB@JFKANBLO@SGXUnregisterHWTransferContextBW@ 100018dc     srvkmbridged:bridged_sgx_bridge.obj
 0001:00000900       ??_C@_0DB@PNGKKIGJ@PVRSRV_BRIDGE_SGX_UNREGISTER_HW_@ 10001900     srvkmbridged:bridged_sgx_bridge.obj
 0001:00000934       ??_C@_0BL@CPDJJJCD@SGXScheduleProcessQueuesBW?$AA@ 10001934     srvkmbridged:bridged_sgx_bridge.obj
 0001:00000950       ??_C@_0CK@FGMOPBHJ@PVRSRV_BRIDGE_SGX_SCHEDULE_PROCE@ 10001950     srvkmbridged:bridged_sgx_bridge.obj
 0001:0000097c       ??_C@_07ECEMPDJM@General?$AA@ 1000197c     srvkmsgx:sgxinit.obj
 0001:00000984       ??_C@_0L@PGEIAGBE@General?5BS?$AA@ 10001984     srvkmsgx:sgxinit.obj
 0001:00000990       ??_C@_07KPJGFCNE@TA?5Data?$AA@ 10001990     srvkmsgx:sgxinit.obj
 0001:00000998       ??_C@_0L@FJNLGMOD@TA?5Data?5BS?$AA@ 10001998     srvkmsgx:sgxinit.obj
 0001:000009a4       ??_C@_0M@HKLGKLCN@Kernel?5Code?$AA@ 100019a4     srvkmsgx:sgxinit.obj
 0001:000009b0       ??_C@_0P@BNNOFOFF@Kernel?5Code?5BS?$AA@ 100019b0     srvkmsgx:sgxinit.obj
 0001:000009c0       ??_C@_0L@OKKEBOLA@KernelData?$AA@ 100019c0     srvkmsgx:sgxinit.obj
 0001:000009cc       ??_C@_0O@ICBOFOND@KernelData?5BS?$AA@ 100019cc     srvkmsgx:sgxinit.obj
 0001:000009dc       ??_C@_0BA@GBONALCE@PixelShaderUSSE?$AA@ 100019dc     srvkmsgx:sgxinit.obj
 0001:000009ec       ??_C@_0BD@EALBFBFE@PixelShaderUSSE?5BS?$AA@ 100019ec     srvkmsgx:sgxinit.obj
 0001:00000a00       ??_C@_0BB@JNKGBMKH@VertexShaderUSSE?$AA@ 10001a00     srvkmsgx:sgxinit.obj
 0001:00000a14       ??_C@_0BE@EHEPOIPP@VertexShaderUSSE?5BS?$AA@ 10001a14     srvkmsgx:sgxinit.obj
 0001:00000a28       ??_C@_0BB@LHDMHLBH@PDSPixelCodeData?$AA@ 10001a28     srvkmsgx:sgxinit.obj
 0001:00000a3c       ??_C@_0BE@LIHHJBPP@PDSPixelCodeData?5BS?$AA@ 10001a3c     srvkmsgx:sgxinit.obj
 0001:00000a50       ??_C@_0BC@JGBCPAPO@PDSVertexCodeData?$AA@ 10001a50     srvkmsgx:sgxinit.obj
 0001:00000a64       ??_C@_0BF@BKOFDGLO@PDSVertexCodeData?5BS?$AA@ 10001a64     srvkmsgx:sgxinit.obj
 0001:00000a7c       ??_C@_0O@MKKIKOIA@CacheCoherent?$AA@ 10001a7c     srvkmsgx:sgxinit.obj
 0001:00000a8c       ??_C@_0BB@ELAGFJPA@CacheCoherent?5BS?$AA@ 10001a8c     srvkmsgx:sgxinit.obj
 0001:00000aa0       ??_C@_0N@BMEHCJPG@3DParameters?$AA@ 10001aa0     srvkmsgx:sgxinit.obj
 0001:00000ab0       ??_C@_0BA@FPANLMKB@3DParameters?5BS?$AA@ 10001ab0     srvkmsgx:sgxinit.obj
 0001:00000d28       ??_C@_0BB@JJLPEHAI@EDMTACodeProfile?$AA@ 10001d28     srvinitsgx:sgxinit.obj
 0001:00000d3c       ??_C@_0CD@IEDMBANE@PowerVREurasia?2HWSettings?2PVRSRV@ 10001d3c     srvinitsgx:sgxinit.obj
 0001:00000d60       ??_C@_06HIJKBDID@SGX?53D?$AA@ 10001d60     srvinitsgx:sgxinit.obj
 0001:00000d68       ??_C@_07BBBHIFGO@SGX?5SPM?$AA@ 10001d68     srvinitsgx:sgxinit.obj
 0001:00000d70       ??_C@_06EIHFDKGD@SGX?5TA?$AA@ 10001d70     srvinitsgx:sgxinit.obj
 0001:00000d78       ??_C@_0M@PCAJPOOC@SGX?5ukernel?$AA@ 10001d78     srvinitsgx:sgxinit.obj
 0001:00000d84       ??_C@_09PJNHAIDJ@CacheCtrl?$AA@ 10001d84     srvinitsgx:sgxinit.obj
 0001:00000d90       ??_C@_0BD@INALHODO@RegBoundReturnZero?$AA@ 10001d90     srvinitsgx:sgxinit.obj
 0001:00000da4       ??_C@_0BD@NECJEAHH@DisableClockGating?$AA@ 10001da4     srvinitsgx:sgxinit.obj
 0001:00000db8       ??_C@_0M@EIHLIIGG@MaxEDMTasks?$AA@ 10001db8     srvinitsgx:sgxinit.obj
 0001:00000dc4       ??_C@_0CC@CFFBCIKF@DisableAlphaCoefficientReOrderin@ 10001dc4     srvinitsgx:sgxinit.obj
 0001:00000e0c       PKM_Deinit                 10001e0c f   pvr_kernel.obj
 0001:00000e44       PKM_Open                   10001e44 f   pvr_kernel.obj
 0001:00000e78       PKM_Close                  10001e78 f   pvr_kernel.obj
 0001:00000ea8       PKM_IOControl              10001ea8 f   pvr_kernel.obj
 0001:00000fbc       PKM_Init                   10001fbc f   pvr_kernel.obj
 0001:00001074       PKM_PowerDown              10002074 f   pvr_kernel.obj
 0001:00001078       PKM_PowerUp                10002078 f   pvr_kernel.obj
 0001:00001104       PVRSRV_BridgeDispatchKM    10002104 f   pvr_bridge_k.obj
 0001:000014c8       PVRSRV_BridgeDispatch      100024c8 f   pvr_bridge_k.obj
 0001:00001c6c       OSAllocMem                 10002c6c f   osfunc_srvkm.obj
 0001:00001cdc       OSFreeMem                  10002cdc f   osfunc_srvkm.obj
 0001:00001d04       QueryUMA                   10002d04 f   osfunc_srvkm.obj
 0001:00001d24       UnMapFromUMAddr            10002d24 f   osfunc_srvkm.obj
 0001:00001dc8       UnmapUserFromKernel        10002dc8 f   osfunc_srvkm.obj
 0001:00001e64       SystemISRWrapper           10002e64 f   osfunc_srvkm.obj
 0001:00001ed4       OSInstallDeviceLISR        10002ed4 f   osfunc_srvkm.obj
 0001:00001fcc       OSUninstallDeviceLISR      10002fcc f   osfunc_srvkm.obj
 0001:0000204c       MISRWrapper                1000304c f   osfunc_srvkm.obj
 0001:0000207c       OSInstallMISR              1000307c f   osfunc_srvkm.obj
 0001:000020fc       OSUninstallMISR            100030fc f   osfunc_srvkm.obj
 0001:00002134       OSScheduleMISR             10003134 f   osfunc_srvkm.obj
 0001:00002158       OSMemCopy                  10003158 f   osfunc_srvkm.obj
 0001:0000215c       OSGetPageSize              1000315c f   osfunc_srvkm.obj
 0001:0000216c       OSCreateResource           1000316c f   osfunc_srvkm.obj
 0001:00002180       OSLockResource             10003180 f   osfunc_srvkm.obj
 0001:000021b0       OSUnlockResource           100031b0 f   osfunc_srvkm.obj
 0001:000021e4       OSIsResourceLocked         100031e4 f   osfunc_srvkm.obj
 0001:00002200       OSGetCurrentProcessIDKM    10003200 f   osfunc_srvkm.obj
 0001:00002204       OSMemSet                   10003204 f   osfunc_srvkm.obj
 0001:00002208       OSMapPhysToLin             10003208 f   osfunc_srvkm.obj
 0001:0000229c       OSUnMapPhysToLin           1000329c f   osfunc_srvkm.obj
 0001:000022ac       OSUnReservePhys            100032ac f   osfunc_srvkm.obj
 0001:000022c8       OSClockus                  100032c8 f   osfunc_srvkm.obj
 0001:000022e0       OSWaitus                   100032e0 f   osfunc_srvkm.obj
 0001:00002320       OSInitEnvData              10003320 f   osfunc_srvkm.obj
 0001:0000234c       OSDeInitEnvData            1000334c f   osfunc_srvkm.obj
 0001:00002354       OSReadHWReg                10003354 f   osfunc_srvkm.obj
 0001:0000235c       OSWriteHWReg               1000335c f   osfunc_srvkm.obj
 0001:00002364       OSSNPrintf                 10003364 f   osfunc_srvkm.obj
 0001:000023d8       OSAddTimer                 100033d8 f   osfunc_srvkm.obj
 0001:00002450       OSRemoveTimer              10003450 f   osfunc_srvkm.obj
 0001:00002498       OSEnableTimer              10003498 f   osfunc_srvkm.obj
 0001:000024e4       OSDisableTimer             100034e4 f   osfunc_srvkm.obj
 0001:00002524       OSEventObjectCreate        10003524 f   osfunc_srvkm.obj
 0001:000025e0       OSEventObjectDestroy       100035e0 f   osfunc_srvkm.obj
 0001:00002624       OSEventObjectWait          10003624 f   osfunc_srvkm.obj
 0001:0000262c       OSEventObjectOpen          1000362c f   osfunc_srvkm.obj
 0001:00002634       OSEventObjectClose         10003634 f   osfunc_srvkm.obj
 0001:0000263c       OSEventObjectSignal        1000363c f   osfunc_srvkm.obj
 0001:00002668       WinCEFormatError           10003668 f   osfunc_srvkm.obj
 0001:0000271c       OSAccessOK                 1000371c f   osfunc_srvkm.obj
 0001:00002788       OSProcHasPrivSrvInit       10003788 f   osfunc_srvkm.obj
 0001:00002790       OSCopyToUser               10003790 f   osfunc_srvkm.obj
 0001:000027b4       OSCopyFromUser             100037b4 f   osfunc_srvkm.obj
 0001:000027d8       OSRegisterMem              100037d8 f   osfunc_srvkm.obj
 0001:00002854       OSUnRegisterMem            10003854 f   osfunc_srvkm.obj
 0001:00002868       OSRegisterDiscontigMem     10003868 f   osfunc_srvkm.obj
 0001:000028c4       OSUnRegisterDiscontigMem   100038c4 f   osfunc_srvkm.obj
 0001:000028d8       OSReserveDiscontigPhys     100038d8 f   osfunc_srvkm.obj
 0001:000029e8       OSUnReserveDiscontigPhys   100039e8 f   osfunc_srvkm.obj
 0001:00002a20       OSAcquirePhysPageAddr      10003a20 f   osfunc_srvkm.obj
 0001:00002adc       OSReleasePhysPageAddr      10003adc f   osfunc_srvkm.obj
 0001:00002b00       OSAllocPages               10003b00 f   osfunc_srvkm.obj
 0001:00002dd0       OSFreePages                10003dd0 f   osfunc_srvkm.obj
 0001:00002e98       MapFromUMAddr              10003e98 f   osfunc_srvkm.obj
 0001:000030b0       MapUserFromKernel          100040b0 f   osfunc_srvkm.obj
 0001:000032c4       OSDestroyResource          100042c4 f   osfunc_srvkm.obj
 0001:000032e0       OSMapLinToCPUPhys          100042e0 f   osfunc_srvkm.obj
 0001:00003350       OSReservePhys              10004350 f   osfunc_srvkm.obj
 0001:000033f0       AtoL                       100043f0 f   registry.obj
 0001:000034f0       OSReadRegistryBinData      100044f0 f   registry.obj
 0001:000036a4       OSReadRegistryDWORDFromString 100046a4 f   registry.obj
 0001:00003760       AllocateDeviceID           10004760 f   srvkmcmn:pvrsrv.obj
 0001:000037a8       FreeDeviceID               100047a8 f   srvkmcmn:pvrsrv.obj
 0001:000037f4       PVRSRVEnumerateDevicesKM   100047f4 f   srvkmcmn:pvrsrv.obj
 0001:00003890       PVRSRVDeInit               10004890 f   srvkmcmn:pvrsrv.obj
 0001:000038d4       PVRSRVRegisterDevice       100048d4 f   srvkmcmn:pvrsrv.obj
 0001:000039a8       PVRSRVInitialiseDevice     100049a8 f   srvkmcmn:pvrsrv.obj
 0001:00003a28       PVRSRVAcquireDeviceDataKM  10004a28 f   srvkmcmn:pvrsrv.obj
 0001:00003ab4       PVRSRVDeinitialiseDevice   10004ab4 f   srvkmcmn:pvrsrv.obj
 0001:00003bb4       PollForValueKM             10004bb4 f   srvkmcmn:pvrsrv.obj
 0001:00003c30       PVRSRVGetMiscInfoKM        10004c30 f   srvkmcmn:pvrsrv.obj
 0001:00004004       PVRSRVSystemLISR           10005004 f   srvkmcmn:pvrsrv.obj
 0001:00004088       PVRSRVMISR                 10005088 f   srvkmcmn:pvrsrv.obj
 0001:000040f4       PVRSRVProcessConnect       100050f4 f   srvkmcmn:pvrsrv.obj
 0001:000040f8       PVRSRVProcessDisconnect    100050f8 f   srvkmcmn:pvrsrv.obj
 0001:000040fc       PVRSRVInit                 100050fc f   srvkmcmn:pvrsrv.obj
 0001:00004194       PVRSRVFinaliseSystem       10005194 f   srvkmcmn:pvrsrv.obj
 0001:000042a8       PVRSRVPerProcessData       100052a8 f   srvkmcmn:perproc.obj
 0001:000042bc       PVRSRVPerProcessDataConnect 100052bc f   srvkmcmn:perproc.obj
 0001:000043d0       PVRSRVPerProcessDataDisconnect 100053d0 f   srvkmcmn:perproc.obj
 0001:00004428       PVRSRVPerProcessDataInit   10005428 f   srvkmcmn:perproc.obj
 0001:00004450       PVRSRVPerProcessDataDeInit 10005450 f   srvkmcmn:perproc.obj
 0001:0000447c       ResManInit                 1000547c f   srvkmcmn:resman.obj
 0001:000044c8       ResManDeInit               100054c8 f   srvkmcmn:resman.obj
 0001:000044f0       PVRSRVResManConnect        100054f0 f   srvkmcmn:resman.obj
 0001:0000458c       ResManRegisterRes          1000558c f   srvkmcmn:resman.obj
 0001:0000463c       ResManFindResourceByPtr    1000563c f   srvkmcmn:resman.obj
 0001:00004784       PVRSRVResManDisconnect     10005784 f   srvkmcmn:resman.obj
 0001:000049b0       ResManFreeResByPtr         100059b0 f   srvkmcmn:resman.obj
 0001:000049cc       ResManFreeResByCriteria    100059cc f   srvkmcmn:resman.obj
 0001:000049f0       ResManDissociateRes        100059f0 f   srvkmcmn:resman.obj
 0001:00004a68       PVRSRVEnumerateDCKM        10005a68 f   srvkmcmn:deviceclass.obj
 0001:00004aec       PVRSRVRegisterDCDeviceKM   10005aec f   srvkmcmn:deviceclass.obj
 0001:00004c90       PVRSRVRemoveDCDeviceKM     10005c90 f   srvkmcmn:deviceclass.obj
 0001:00004d60       PVRSRVRegisterBCDeviceKM   10005d60 f   srvkmcmn:deviceclass.obj
 0001:00004f00       PVRSRVRemoveBCDeviceKM     10005f00 f   srvkmcmn:deviceclass.obj
 0001:00004fc8       PVRSRVCloseDCDeviceKM      10005fc8 f   srvkmcmn:deviceclass.obj
 0001:00005030       PVRSRVOpenDCDeviceKM       10006030 f   srvkmcmn:deviceclass.obj
 0001:0000519c       PVRSRVEnumDCFormatsKM      1000619c f   srvkmcmn:deviceclass.obj
 0001:000051dc       PVRSRVEnumDCDimsKM         100061dc f   srvkmcmn:deviceclass.obj
 0001:0000521c       PVRSRVGetDCSystemBufferKM  1000621c f   srvkmcmn:deviceclass.obj
 0001:000052a4       PVRSRVGetDCInfoKM          100062a4 f   srvkmcmn:deviceclass.obj
 0001:000052fc       PVRSRVDestroyDCSwapChainKM 100062fc f   srvkmcmn:deviceclass.obj
 0001:000053a0       PVRSRVCreateDCSwapChainKM  100063a0 f   srvkmcmn:deviceclass.obj
 0001:00005620       PVRSRVSetDCDstRectKM       10006620 f   srvkmcmn:deviceclass.obj
 0001:0000565c       PVRSRVSetDCSrcRectKM       1000665c f   srvkmcmn:deviceclass.obj
 0001:00005698       PVRSRVSetDCDstColourKeyKM  10006698 f   srvkmcmn:deviceclass.obj
 0001:000056d4       PVRSRVSetDCSrcColourKeyKM  100066d4 f   srvkmcmn:deviceclass.obj
 0001:00005710       PVRSRVGetDCBuffersKM       10006710 f   srvkmcmn:deviceclass.obj
 0001:000057ac       PVRSRVSwapToDCBufferKM     100067ac f   srvkmcmn:deviceclass.obj
 0001:00005968       PVRSRVSwapToDCSystemKM     10006968 f   srvkmcmn:deviceclass.obj
 0001:00005ab0       PVRSRVRegisterSystemISRHandler 10006ab0 f   srvkmcmn:deviceclass.obj
 0001:00005b0c       PVRSRVSetDCState           10006b0c f   srvkmcmn:deviceclass.obj
 0001:00005b74       PVRGetDisplayClassJTable   10006b74 f   srvkmcmn:deviceclass.obj
 0001:00005be0       PVRSRVCloseBCDeviceKM      10006be0 f   srvkmcmn:deviceclass.obj
 0001:00005c8c       PVRSRVOpenBCDeviceKM       10006c8c f   srvkmcmn:deviceclass.obj
 0001:00005f14       PVRSRVGetBCInfoKM          10006f14 f   srvkmcmn:deviceclass.obj
 0001:00005f4c       PVRSRVGetBCBufferKM        10006f4c f   srvkmcmn:deviceclass.obj
 0001:00005f90       PVRGetBufferClassJTable    10006f90 f   srvkmcmn:deviceclass.obj
 0001:00006534       PVRSRVAllocHandle          10007534 f   srvkmcmn:handle.obj
 0001:0000661c       PVRSRVAllocSubHandle       1000761c f   srvkmcmn:handle.obj
 0001:000067cc       PVRSRVFindHandle           100077cc f   srvkmcmn:handle.obj
 0001:00006810       PVRSRVLookupHandleAnyType  10007810 f   srvkmcmn:handle.obj
 0001:00006854       PVRSRVLookupHandle         10007854 f   srvkmcmn:handle.obj
 0001:00006884       PVRSRVLookupSubHandle      10007884 f   srvkmcmn:handle.obj
 0001:00006910       PVRSRVGetParentHandle      10007910 f   srvkmcmn:handle.obj
 0001:00006940       PVRSRVLookupAndReleaseHandle 10007940 f   srvkmcmn:handle.obj
 0001:00006978       PVRSRVReleaseHandle        10007978 f   srvkmcmn:handle.obj
 0001:000069ac       PVRSRVNewHandleBatch       100079ac f   srvkmcmn:handle.obj
 0001:00006ab4       PVRSRVCommitHandleBatch    10007ab4 f   srvkmcmn:handle.obj
 0001:00006abc       PVRSRVReleaseHandleBatch   10007abc f   srvkmcmn:handle.obj
 0001:00006ac4       PVRSRVPurgeHandles         10007ac4 f   srvkmcmn:handle.obj
 0001:00006c6c       PVRSRVFreeHandleBase       10007c6c f   srvkmcmn:handle.obj
 0001:00006c70       PVRSRVHandleDeInit         10007c70 f   srvkmcmn:handle.obj
 0001:00006ca4       PVRSRVAllocHandleBase      10007ca4 f   srvkmcmn:handle.obj
 0001:00006d4c       PVRSRVHandleInit           10007d4c f   srvkmcmn:handle.obj
 0001:00006db0       PVRSRVSetInitServerState   10007db0 f   srvkmcmn:power.obj
 0001:00006dfc       PVRSRVGetInitServerState   10007dfc f   srvkmcmn:power.obj
 0001:00006e3c       PVRSRVPowerUnlock          10007e3c f   srvkmcmn:power.obj
 0001:00006fb0       PVRSRVSystemPostPowerStateKM 10007fb0 f   srvkmcmn:power.obj
 0001:00007070       PVRSRVRemovePowerDevice    10008070 f   srvkmcmn:power.obj
 0001:000070e0       PVRSRVIsDevicePowered      100080e0 f   srvkmcmn:power.obj
 0001:00007160       PVRSRVPowerLock            10008160 f   srvkmcmn:power.obj
 0001:000071fc       PVRSRVSetDevicePowerStateKM 100081fc f   srvkmcmn:power.obj
 0001:00007294       PVRSRVSystemPrePowerStateKM 10008294 f   srvkmcmn:power.obj
 0001:00007348       PVRSRVSetPowerStateKM      10008348 f   srvkmcmn:power.obj
 0001:0000739c       PVRSRVRegisterPowerDevice  1000839c f   srvkmcmn:power.obj
 0001:00007ef4       RA_Create                  10008ef4 f   srvkmcmn:ra.obj
 0001:00008090       RA_Delete                  10009090 f   srvkmcmn:ra.obj
 0001:0000812c       RA_TestDelete              1000912c f   srvkmcmn:ra.obj
 0001:0000815c       RA_Alloc                   1000915c f   srvkmcmn:ra.obj
 0001:000082d8       RA_Free                    100092d8 f   srvkmcmn:ra.obj
 0001:00008314       RA_GetStats                10009314 f   srvkmcmn:ra.obj
 0001:000087b4       BM_DestroyContext          100097b4 f   srvkmcmn:buffer_manager.obj
 0001:00008940       BM_CreateContext           10009940 f   srvkmcmn:buffer_manager.obj
 0001:00008b2c       BM_DestroyHeap             10009b2c f   srvkmcmn:buffer_manager.obj
 0001:00008bb4       BM_HandleToCpuVaddr        10009bb4 f   srvkmcmn:buffer_manager.obj
 0001:00008bc4       BM_HandleToDevVaddr        10009bc4 f   srvkmcmn:buffer_manager.obj
 0001:00008bdc       BM_HandleToOSMemHandle     10009bdc f   srvkmcmn:buffer_manager.obj
 0001:00009098       BM_GetPhysPageAddr         1000a098 f   srvkmcmn:buffer_manager.obj
 0001:00009110       BM_GetMMUContextFromMemContext 1000a110 f   srvkmcmn:buffer_manager.obj
 0001:00009118       BM_GetDeviceNode           1000a118 f   srvkmcmn:buffer_manager.obj
 0001:0000972c       BM_CreateHeap              1000a72c f   srvkmcmn:buffer_manager.obj
 0001:00009924       BM_Alloc                   1000a924 f   srvkmcmn:buffer_manager.obj
 0001:00009a10       BM_Wrap                    1000aa10 f   srvkmcmn:buffer_manager.obj
 0001:00009bf0       BM_Free                    1000abf0 f   srvkmcmn:buffer_manager.obj
 0001:00009c78       PVRSRVCreateCommandQueueKM 1000ac78 f   srvkmcmn:queue.obj
 0001:00009df4       PVRSRVDestroyCommandQueueKM 1000adf4 f   srvkmcmn:queue.obj
 0001:00009f24       PVRSRVGetQueueSpaceKM      1000af24 f   srvkmcmn:queue.obj
 0001:00009fd4       PVRSRVInsertCommandKM      1000afd4 f   srvkmcmn:queue.obj
 0001:0000a130       PVRSRVSubmitCommandKM      1000b130 f   srvkmcmn:queue.obj
 0001:0000a1c0       PVRSRVProcessCommand       1000b1c0 f   srvkmcmn:queue.obj
 0001:0000a3d0       PVRSRVProcessQueues        1000b3d0 f   srvkmcmn:queue.obj
 0001:0000a4f4       PVRSRVCommandCompleteCallbacks 1000b4f4 f   srvkmcmn:queue.obj
 0001:0000a538       PVRSRVRegisterCmdProcListKM 1000b538 f   srvkmcmn:queue.obj
 0001:0000a6e8       PVRSRVRemoveCmdProcListKM  1000b6e8 f   srvkmcmn:queue.obj
 0001:0000a794       PVRSRVCommandCompleteKM    1000b794 f   srvkmcmn:queue.obj
 0001:0000a84c       HASH_Func_Default          1000b84c f   srvkmcmn:hash.obj
 0001:0000a88c       HASH_Key_Comp_Default      1000b88c f   srvkmcmn:hash.obj
 0001:0000a9f8       HASH_Create_Extended       1000b9f8 f   srvkmcmn:hash.obj
 0001:0000aae0       HASH_Create                1000bae0 f   srvkmcmn:hash.obj
 0001:0000aaf8       HASH_Delete                1000baf8 f   srvkmcmn:hash.obj
 0001:0000ab30       HASH_Insert_Extended       1000bb30 f   srvkmcmn:hash.obj
 0001:0000ac20       HASH_Insert                1000bc20 f   srvkmcmn:hash.obj
 0001:0000ac38       HASH_Remove_Extended       1000bc38 f   srvkmcmn:hash.obj
 0001:0000ad28       HASH_Remove                1000bd28 f   srvkmcmn:hash.obj
 0001:0000ad40       HASH_Retrieve_Extended     1000bd40 f   srvkmcmn:hash.obj
 0001:0000add0       HASH_Retrieve              1000bdd0 f   srvkmcmn:hash.obj
 0001:0000ade8       PVRSRVGetDeviceMemHeapsKM  1000bde8 f   srvkmcmn:devicemem.obj
 0001:0000ae90       PVRSRVCreateDeviceMemContextKM 1000be90 f   srvkmcmn:devicemem.obj
 0001:0000afa4       PVRSRVDestroyDeviceMemContextKM 1000bfa4 f   srvkmcmn:devicemem.obj
 0001:0000afb0       PVRSRVGetDeviceMemHeapInfoKM 1000bfb0 f   srvkmcmn:devicemem.obj
 0001:0000b1f8       PVRSRVAllocSyncInfoKM      1000c1f8 f   srvkmcmn:devicemem.obj
 0001:0000b308       PVRSRVFreeSyncInfoKM       1000c308 f   srvkmcmn:devicemem.obj
 0001:0000b3f0       PVRSRVFreeDeviceMemKM      1000c3f0 f   srvkmcmn:devicemem.obj
 0001:0000b434       PVRSRVAllocDeviceMemKM     1000c434 f   srvkmcmn:devicemem.obj
 0001:0000b524       PVRSRVDissociateDeviceMemKM 1000c524 f   srvkmcmn:devicemem.obj
 0001:0000b544       PVRSRVGetFreeDeviceMemKM   1000c544 f   srvkmcmn:devicemem.obj
 0001:0000b54c       PVRSRVUnwrapExtMemoryKM    1000c54c f   srvkmcmn:devicemem.obj
 0001:0000b5e0       PVRSRVWrapExtMemoryKM      1000c5e0 f   srvkmcmn:devicemem.obj
 0001:0000b90c       PVRSRVUnmapDeviceMemoryKM  1000c90c f   srvkmcmn:devicemem.obj
 0001:0000b9a8       PVRSRVMapDeviceMemoryKM    1000c9a8 f   srvkmcmn:devicemem.obj
 0001:0000bcac       PVRSRVUnmapDeviceClassMemoryKM 1000ccac f   srvkmcmn:devicemem.obj
 0001:0000bccc       PVRSRVMapDeviceClassMemoryKM 1000cccc f   srvkmcmn:devicemem.obj
 0001:0000bf10       SrvInit                    1000cf10 f   srvinitcommon:srvinit.obj
 0001:0000bfc0       PVRSRVCallocUserModeMem    1000cfc0 f   srvclkm:srvclient_wince.obj
 0001:0000bfcc       PVRSRVMemCopy              1000cfcc f   srvclkm:srvclient_wince.obj
 0001:0000bfd0       PVRSRVMemSet               1000cfd0 f   srvclkm:srvclient_wince.obj
 0001:0000bfd4       PVRSRVBridgeCall           1000cfd4 f   srvclkm:pvr_bridge_clientkm.obj
 0001:0000c0d4       SetJTable                  1000d0d4 f   srvclkm:pvr_bridge_clientkm.obj
 0001:0000c0f4       PVRSRVInitSrvConnect       1000d0f4 f   srvclkm:pvr_glue.obj
 0001:0000c154       PVRSRVInitSrvDisconnect    1000d154 f   srvclkm:pvr_glue.obj
 0001:0000c1b4       PVRSRVAllocDeviceMem       1000d1b4 f   srvclkm:pvr_glue.obj
 0001:0000c2c4       PVRSRVUnrefDeviceMem       1000d2c4 f   srvclkm:pvr_glue.obj
 0001:0000c304       PVRSRVEnumerateDevices     1000d304 f   srvclkm:bridged_pvr_glue.obj
 0001:0000c3b0       PVRSRVAcquireDeviceData    1000d3b0 f   srvclkm:bridged_pvr_glue.obj
 0001:0000c434       PVRSRVAllocUserModeMem     1000d434 f   srvclkm:osfnex_clientkm.obj
 0001:0000c440       PVRSRVFreeUserModeMem      1000d440 f   srvclkm:osfnex_clientkm.obj
 0001:0000c444       SysDeinitialise            1000d444 f   system:sysconfig.obj
 0001:0000c4dc       SysGetDeviceMemoryMap      1000d4dc f   system:sysconfig.obj
 0001:0000c4f4       SysCpuPAddrToDevPAddr      1000d4f4 f   system:sysconfig.obj
 0001:0000c4fc       SysSysPAddrToCpuPAddr      1000d4fc f   system:sysconfig.obj
 0001:0000c504       SysCpuPAddrToSysPAddr      1000d504 f   system:sysconfig.obj
 0001:0000c50c       SysSysPAddrToDevPAddr      1000d50c f   system:sysconfig.obj
 0001:0000c514       SysDevPAddrToSysPAddr      1000d514 f   system:sysconfig.obj
 0001:0000c51c       SysRegisterExternalDevice  1000d51c f   system:sysconfig.obj
 0001:0000c520       SysRemoveExternalDevice    1000d520 f   system:sysconfig.obj
 0001:0000c524       SysGetInterruptSource      1000d524 f   system:sysconfig.obj
 0001:0000c52c       SysClearInterrupts         1000d52c f   system:sysconfig.obj
 0001:0000c530       SysSystemPrePowerState     1000d530 f   system:sysconfig.obj
 0001:0000c538       SysSystemPostPowerState    1000d538 f   system:sysconfig.obj
 0001:0000c540       SysDevicePrePowerState     1000d540 f   system:sysconfig.obj
 0001:0000c548       SysDevicePostPowerState    1000d548 f   system:sysconfig.obj
 0001:0000c550       SysOEMFunction             1000d550 f   system:sysconfig.obj
 0001:0000c574       SysInitialise              1000d574 f   system:sysconfig.obj
 0001:0000c81c       SysFinalise                1000d81c f   system:sysconfig.obj
 0001:0000e684       DummyBW                    1000f684 f   srvkmbridged:bridged_pvr_bridge.obj
 0001:0000e68c       _SetDispatchTableEntry     1000f68c f   srvkmbridged:bridged_pvr_bridge.obj
 0001:0000e8d0       CommonBridgeInit           1000f8d0 f   srvkmbridged:bridged_pvr_bridge.obj
 0001:0000ebf0       BridgedDispatchKM          1000fbf0 f   srvkmbridged:bridged_pvr_bridge.obj
 0001:0000ff2c       SetSGXDispatchTableEntry   10010f2c f   srvkmbridged:bridged_sgx_bridge.obj
 0001:000101dc       WaitForSingleObject        100111dc f   coredll:COREDLL.dll
 0001:000101ec       ReleaseMutex               100111ec f   coredll:COREDLL.dll
 0001:000101fc       CloseHandle                100111fc f   coredll:COREDLL.dll
 0001:0001020c       CreateMutexW               1001120c f   coredll:COREDLL.dll
 0001:0001021c       __GetUserKData             1001121c f   coredll:COREDLL.dll
 0001:0001022c       NKDbgPrintfW               1001122c f   coredll:COREDLL.dll
 0001:0001023c       GetDirectCallerProcessId   1001123c f   coredll:COREDLL.dll
 0001:0001024c       KernelLibIoControl         1001124c f   coredll:COREDLL.dll
 0001:0001025c       EventModify                1001125c f   coredll:COREDLL.dll
 0001:0001026c       LockPages                  1001126c f   coredll:COREDLL.dll
 0001:0001027c       UnlockPages                1001127c f   coredll:COREDLL.dll
 0001:0001028c       VirtualFreeEx              1001128c f   coredll:COREDLL.dll
 0001:0001029c       InterruptDone              1001129c f   coredll:COREDLL.dll
 0001:000102ac       CeSetThreadPriority        100112ac f   coredll:COREDLL.dll
 0001:000102bc       InterruptDisable           100112bc f   coredll:COREDLL.dll
 0001:000102cc       CreateThread               100112cc f   coredll:COREDLL.dll
 0001:000102dc       InterruptInitialize        100112dc f   coredll:COREDLL.dll
 0001:000102ec       CreateEventW               100112ec f   coredll:COREDLL.dll
 0001:000102fc       KernelIoControl            100112fc f   coredll:COREDLL.dll
 0001:0001030c       TerminateThread            1001130c f   coredll:COREDLL.dll
 0001:0001031c       RegCloseKey                1001131c f   coredll:COREDLL.dll
 0001:0001032c       RegQueryValueExW           1001132c f   coredll:COREDLL.dll
 0001:0001033c       RegOpenKeyExW              1001133c f   coredll:COREDLL.dll
 0001:0001034c       InterlockedCompareExchange 1001134c f   coredll:COREDLL.dll
 0001:0001035c       GetCallerVMProcessId       1001135c f   coredll:COREDLL.dll
 0001:0001036c       GetTickCount               1001136c f   coredll:COREDLL.dll
 0001:0001037c       LocalFree                  1001137c f   coredll:COREDLL.dll
 0001:0001038c       FormatMessageW             1001138c f   coredll:COREDLL.dll
 0001:0001039c       IsBadWritePtr              1001139c f   coredll:COREDLL.dll
 0001:000103ac       IsBadReadPtr               100113ac f   coredll:COREDLL.dll
 0001:000103bc       VirtualCopy                100113bc f   coredll:COREDLL.dll
 0001:000103cc       VirtualAlloc               100113cc f   coredll:COREDLL.dll
 0001:000103dc       VirtualFree                100113dc f   coredll:COREDLL.dll
 0001:000103ec       GetLastError               100113ec f   coredll:COREDLL.dll
 0001:000103fc       VirtualAllocEx             100113fc f   coredll:COREDLL.dll
 0001:0001040c       VirtualAllocCopyEx         1001140c f   coredll:COREDLL.dll
 0001:0001041c       VirtualCopyEx              1001141c f   coredll:COREDLL.dll
 0001:0001042c       WideCharToMultiByte        1001142c f   coredll:COREDLL.dll
 0001:0001043c       DeviceIoControl            1001143c f   coredll:COREDLL.dll
 0001:0001044c       CreateFileW                1001144c f   coredll:COREDLL.dll
 0001:0001045c       LocalAlloc                 1001145c f   coredll:COREDLL.dll
 0001:0001046c       MmMapIoSpace               1001146c f   CEDDK:CEDDK.dll
 0001:0001047c       MmUnmapIoSpace             1001147c f   CEDDK:CEDDK.dll
 0001:0001048c       DllMain                    1001148c f   corelib0:dllmain.obj
 0001:000105a8       _DllMainCRTStartup         100115a8 f   corelib0:pegdmain.obj
 0001:000105d8       __GSHandlerCheckCommon     100115d8 f   corelib0:gshandler.obj
 0001:00010614       __GSHandlerCheck           10011614 f   corelib0:gshandler.obj
 0001:00010638       __security_init_cookie     10011638 f   corelib0:seccinit.obj
 0001:00010694       __security_check_cookie    10011694 f   corelib0:armsecgs.obj
 0001:000106a8       __gsfailure                100116a8 f   corelib0:armsecgs.obj
 0001:000107b4       _cexit                     100117b4 f   corelib0:cexit.obj
 0001:000107d0       _initterm                  100117d0 f   corelib0:crt0dat.obj
 0001:00010804       _cinit                     10011804 f   corelib0:crt0dat.obj
 0001:00010838       memset                     10011838 f   corelib1:COREDLL.dll
 0001:00010848       free                       10011848 f   corelib1:COREDLL.dll
 0001:00010858       malloc                     10011858 f   corelib1:COREDLL.dll
 0001:00010868       memcpy                     10011868 f   corelib1:COREDLL.dll
 0001:00010878       vsprintf                   10011878 f   corelib1:COREDLL.dll
 0001:00010888       swprintf                   10011888 f   corelib1:COREDLL.dll
 0001:00010898       _snprintf                  10011898 f   corelib1:COREDLL.dll
 0001:000108a8       strncpy                    100118a8 f   corelib1:COREDLL.dll
 0001:000108b8       __C_specific_handler       100118b8 f   corelib1:COREDLL.dll
 0001:000108c8       strcat                     100118c8 f   corelib1:COREDLL.dll
 0001:000108d8       strlen                     100118d8 f   corelib1:COREDLL.dll
 0001:000108e8       calloc                     100118e8 f   corelib1:COREDLL.dll
 0001:000108f8       _XcptFilter                100118f8 f   corelib1:COREDLL.dll
 0001:00010908       __security_gen_cookie2     10011908 f   corelib1:COREDLL.dll
 0001:00010918       __report_gsfailure         10011918 f   corelib1:COREDLL.dll
 0001:00010a9c       SGXInitialise              10011a9c f   srvkmsgx:sgxinit.obj
 0001:00010bc0       SGXDeinitialise            10011bc0 f   srvkmsgx:sgxinit.obj
 0001:00010d1c       SGXGetInfoForSrvinitKM     10011d1c f   srvkmsgx:sgxinit.obj
 0001:00010d40       DevInitSGXPart2KM          10011d40 f   srvkmsgx:sgxinit.obj
 0001:00010fb4       SGXOSTimer                 10011fb4 f   srvkmsgx:sgxinit.obj
 0001:000110d4       SGX_ISRHandler             100120d4 f   srvkmsgx:sgxinit.obj
 0001:00011140       SGX_MISRHandler            10012140 f   srvkmsgx:sgxinit.obj
 0001:000111cc       SGXGetClientInfoKM         100121cc f   srvkmsgx:sgxinit.obj
 0001:000112e0       SGXGetMiscInfoKM           100122e0 f   srvkmsgx:sgxinit.obj
 0001:00011380       SGXDevInitCompatCheck      10012380 f   srvkmsgx:sgxinit.obj
 0001:00011400       SGXRegisterDevice          10012400 f   srvkmsgx:sgxinit.obj
 0001:0001182c       SGXPostActivePowerEvent    1001282c f   srvkmsgx:sgxutils.obj
 0001:00011868       SGXTestActivePowerEvent    10012868 f   srvkmsgx:sgxutils.obj
 0001:000118d4       SGXScheduleCCBCommand      100128d4 f   srvkmsgx:sgxutils.obj
 0001:00011a08       SGXScheduleCCBCommandKM    10012a08 f   srvkmsgx:sgxutils.obj
 0001:00011aa8       SGXScheduleProcessQueuesKM 10012aa8 f   srvkmsgx:sgxutils.obj
 0001:00011b1c       SGXIsDevicePowered         10012b1c f   srvkmsgx:sgxutils.obj
 0001:00011b24       SGXGetInternalDevInfoKM    10012b24 f   srvkmsgx:sgxutils.obj
 0001:00011b48       SGXCleanupRequest          10012b48 f   srvkmsgx:sgxutils.obj
 0001:00011c70       SGXRegisterHWRenderContextKM 10012c70 f   srvkmsgx:sgxutils.obj
 0001:00011d20       SGXUnregisterHWRenderContextKM 10012d20 f   srvkmsgx:sgxutils.obj
 0001:00011d3c       SGXRegisterHWTransferContextKM 10012d3c f   srvkmsgx:sgxutils.obj
 0001:00011dec       SGXUnregisterHWTransferContextKM 10012dec f   srvkmsgx:sgxutils.obj
 0001:00011e08       SGX2DQueryBlitsCompleteKM  10012e08 f   srvkmsgx:sgxutils.obj
 0001:00011eac       SGXFlushHWRenderTargetKM   10012eac f   srvkmsgx:sgxutils.obj
 0001:00011ec8       SGXDoKickKM                10012ec8 f   srvkmsgx:sgxkick.obj
 0001:00012200       SGXSubmitTransferKM        10013200 f   srvkmsgx:sgxtransfer.obj
 0001:000124e0       SGXUnrefSharedPBDescKM     100134e0 f   srvkmsgx:pb.obj
 0001:000124e4       SGXAddSharedPBDescKM       100134e4 f   srvkmsgx:pb.obj
 0001:00012754       SGXFindSharedPBDescKM      10013754 f   srvkmsgx:pb.obj
 0001:000129f4       SGXStartTimer              100139f4 f   srvkmsgx:sgxpower.obj
 0001:00012bdc       SGXPrePowerStateExt        10013bdc f   srvkmsgx:sgxpower.obj
 0001:00012c24       SGXPostPowerStateExt       10013c24 f   srvkmsgx:sgxpower.obj
 0001:00012c6c       SGXPreClockSpeedChange     10013c6c f   srvkmsgx:sgxpower.obj
 0001:00012c9c       SGXPostClockSpeedChange    10013c9c f   srvkmsgx:sgxpower.obj
 0001:00012e00       SGXReset                   10013e00 f   srvkmsgx:sgxreset.obj
 0001:0001346c       MMU_Initialise             1001446c f   srvkmsgx:mmu.obj
 0001:00013628       MMU_Finalise               10014628 f   srvkmsgx:mmu.obj
 0001:0001372c       MMU_InsertHeap             1001472c f   srvkmsgx:mmu.obj
 0001:000137a8       MMU_FreePageTables         100147a8 f   srvkmsgx:mmu.obj
 0001:0001388c       MMU_Create                 1001488c f   srvkmsgx:mmu.obj
 0001:000139e0       MMU_Delete                 100149e0 f   srvkmsgx:mmu.obj
 0001:00013a58       MMU_Alloc                  10014a58 f   srvkmsgx:mmu.obj
 0001:00013ad8       MMU_Free                   10014ad8 f   srvkmsgx:mmu.obj
 0001:00013ba0       MMU_MapScatter             10014ba0 f   srvkmsgx:mmu.obj
 0001:00013c08       MMU_MapPages               10014c08 f   srvkmsgx:mmu.obj
 0001:00013c84       MMU_MapShadow              10014c84 f   srvkmsgx:mmu.obj
 0001:00013d28       MMU_UnmapPages             10014d28 f   srvkmsgx:mmu.obj
 0001:00013db4       MMU_GetPhysPageAddr        10014db4 f   srvkmsgx:mmu.obj
 0001:00013dfc       MMU_GetPDDevPAddr          10014dfc f   srvkmsgx:mmu.obj
 0001:00013e0c       MMU_BIFResetPDAlloc        10014e0c f   srvkmsgx:mmu.obj
 0001:00013f84       MMU_BIFResetPDFree         10014f84 f   srvkmsgx:mmu.obj
 0001:00015010       SGXInit                    10016010 f   srvinitsgx:sgxinit.obj
 0001:000151fc       PVRSRVAllocSharedSysMemoryKM 100161fc f   srvkmcmn:mem.obj
 0001:000152dc       PVRSRVFreeSharedSysMemoryKM 100162dc f   srvkmcmn:mem.obj
 0001:000152f4       PVRSRVDissociateMemFromResmanKM 100162f4 f   srvkmcmn:mem.obj
 0001:00015334       SGXGetInfoForSrvInit       10016334 f   srvclkm:bridged_sgx_glue.obj
 0001:000153a4       SGXDevInitPart2            100163a4 f   srvclkm:bridged_sgx_glue.obj
 0001:000155cc       DisableThreadLibraryCalls  100165cc f   coredll:COREDLL.dll
 0001:000155dc       TerminateProcess           100165dc f   coredll:COREDLL.dll
 0001:00015620       __IMPORT_DESCRIPTOR_COREDLL 10016620     coredll:COREDLL.dll
 0001:00015634       __IMPORT_DESCRIPTOR_CEDDK  10016634     CEDDK:CEDDK.dll
 0001:00015648       __NULL_IMPORT_DESCRIPTOR   10016648     coredll:COREDLL.dll
 0002:00000000       __imp_MmMapIoSpace         10017000     CEDDK:CEDDK.dll
 0002:00000004       __imp_MmUnmapIoSpace       10017004     CEDDK:CEDDK.dll
 0002:00000008       \177CEDDK_NULL_THUNK_DATA  10017008     CEDDK:CEDDK.dll
 0002:0000000c       __imp_CreateMutexW         1001700c     coredll:COREDLL.dll
 0002:00000010       __imp___GetUserKData       10017010     coredll:COREDLL.dll
 0002:00000014       __imp_NKDbgPrintfW         10017014     coredll:COREDLL.dll
 0002:00000018       __imp_GetDirectCallerProcessId 10017018     coredll:COREDLL.dll
 0002:0000001c       __imp_KernelLibIoControl   1001701c     coredll:COREDLL.dll
 0002:00000020       __imp_EventModify          10017020     coredll:COREDLL.dll
 0002:00000024       __imp_LockPages            10017024     coredll:COREDLL.dll
 0002:00000028       __imp_UnlockPages          10017028     coredll:COREDLL.dll
 0002:0000002c       __imp_VirtualFreeEx        1001702c     coredll:COREDLL.dll
 0002:00000030       __imp_InterruptDone        10017030     coredll:COREDLL.dll
 0002:00000034       __imp_CeSetThreadPriority  10017034     coredll:COREDLL.dll
 0002:00000038       __imp_InterruptDisable     10017038     coredll:COREDLL.dll
 0002:0000003c       __imp_CreateThread         1001703c     coredll:COREDLL.dll
 0002:00000040       __imp_InterruptInitialize  10017040     coredll:COREDLL.dll
 0002:00000044       __imp_CreateEventW         10017044     coredll:COREDLL.dll
 0002:00000048       __imp_KernelIoControl      10017048     coredll:COREDLL.dll
 0002:0000004c       __imp_TerminateThread      1001704c     coredll:COREDLL.dll
 0002:00000050       __imp_RegCloseKey          10017050     coredll:COREDLL.dll
 0002:00000054       __imp_RegQueryValueExW     10017054     coredll:COREDLL.dll
 0002:00000058       __imp_RegOpenKeyExW        10017058     coredll:COREDLL.dll
 0002:0000005c       __imp_InterlockedCompareExchange 1001705c     coredll:COREDLL.dll
 0002:00000060       __imp_CloseHandle          10017060     coredll:COREDLL.dll
 0002:00000064       __imp_GetTickCount         10017064     coredll:COREDLL.dll
 0002:00000068       __imp_LocalFree            10017068     coredll:COREDLL.dll
 0002:0000006c       __imp_FormatMessageW       1001706c     coredll:COREDLL.dll
 0002:00000070       __imp_IsBadWritePtr        10017070     coredll:COREDLL.dll
 0002:00000074       __imp_IsBadReadPtr         10017074     coredll:COREDLL.dll
 0002:00000078       __imp_VirtualCopy          10017078     coredll:COREDLL.dll
 0002:0000007c       __imp_VirtualAlloc         1001707c     coredll:COREDLL.dll
 0002:00000080       __imp_VirtualFree          10017080     coredll:COREDLL.dll
 0002:00000084       __imp_GetLastError         10017084     coredll:COREDLL.dll
 0002:00000088       __imp_VirtualAllocEx       10017088     coredll:COREDLL.dll
 0002:0000008c       __imp_VirtualAllocCopyEx   1001708c     coredll:COREDLL.dll
 0002:00000090       __imp_VirtualCopyEx        10017090     coredll:COREDLL.dll
 0002:00000094       __imp_WideCharToMultiByte  10017094     coredll:COREDLL.dll
 0002:00000098       __imp_DeviceIoControl      10017098     coredll:COREDLL.dll
 0002:0000009c       __imp_CreateFileW          1001709c     coredll:COREDLL.dll
 0002:000000a0       __imp_LocalAlloc           100170a0     coredll:COREDLL.dll
 0002:000000a4       __imp_ReleaseMutex         100170a4     coredll:COREDLL.dll
 0002:000000a8       __imp_GetCallerVMProcessId 100170a8     coredll:COREDLL.dll
 0002:000000ac       __imp_WaitForSingleObject  100170ac     coredll:COREDLL.dll
 0002:000000b0       __imp_memset               100170b0     corelib1:COREDLL.dll
 0002:000000b4       __imp_free                 100170b4     corelib1:COREDLL.dll
 0002:000000b8       __imp_malloc               100170b8     corelib1:COREDLL.dll
 0002:000000bc       __imp_memcpy               100170bc     corelib1:COREDLL.dll
 0002:000000c0       __imp_vsprintf             100170c0     corelib1:COREDLL.dll
 0002:000000c4       __imp_swprintf             100170c4     corelib1:COREDLL.dll
 0002:000000c8       __imp__snprintf            100170c8     corelib1:COREDLL.dll
 0002:000000cc       __imp_strncpy              100170cc     corelib1:COREDLL.dll
 0002:000000d0       __imp___C_specific_handler 100170d0     corelib1:COREDLL.dll
 0002:000000d4       __imp___rt_udiv            100170d4     corelib1:COREDLL.dll
 0002:000000d8       __imp_strcat               100170d8     corelib1:COREDLL.dll
 0002:000000dc       __imp_strlen               100170dc     corelib1:COREDLL.dll
 0002:000000e0       __imp_calloc               100170e0     corelib1:COREDLL.dll
 0002:000000e4       __imp__XcptFilter          100170e4     corelib1:COREDLL.dll
 0002:000000e8       __imp___security_gen_cookie2 100170e8     corelib1:COREDLL.dll
 0002:000000ec       __imp___report_gsfailure   100170ec     corelib1:COREDLL.dll
 0002:000000f0       __imp_DisableThreadLibraryCalls 100170f0     coredll:COREDLL.dll
 0002:000000f4       __imp_TerminateProcess     100170f4     coredll:COREDLL.dll
 0002:000000f8       \177COREDLL_NULL_THUNK_DATA 100170f8     coredll:COREDLL.dll
 0002:00000100       gui32ClientInKernelMode    10017100     pvr_kernel.obj
 0002:00000104       gPVRDebugLevel             10017104     pvr_debug.obj
 0002:00000108       version_string             10017108     system:sysconfig.obj
 0002:00000120       __security_cookie          10017120     corelib0:seccinit.obj
 0002:00000124       __security_cookie_complement 10017124     corelib0:seccinit.obj
 0002:00000128       pbuKernelProgram           10017128     srvinitsgx:sgxinit.obj
 0002:00003e48       pbuKernelTAProgram         1001ae48     srvinitsgx:sgxinit.obj
 0002:000075d8       pbuKernelSPMProgram        1001e5d8     srvinitsgx:sgxinit.obj
 0002:0000a698       pbuKernel3DProgram         10021698     srvinitsgx:sgxinit.obj
 0002:0000f2d0       ui32uKernelProgramSizes    100262d0     srvinitsgx:sgxinit.obj
 0002:0000f2d4       ui32uKernelTAProgramSizes  100262d4     srvinitsgx:sgxinit.obj
 0002:0000f2d8       ui32uKernel3DProgramSizes  100262d8     srvinitsgx:sgxinit.obj
 0002:0000f2dc       pbuKernelProgramBlocks     100262dc     srvinitsgx:sgxinit.obj
 0002:0000f2e0       pbuKernelTAProgramBlocks   100262e0     srvinitsgx:sgxinit.obj
 0002:0000f2e4       pbuKernel3DProgramBlocks   100262e4     srvinitsgx:sgxinit.obj
 0002:0000f2e8       ui32uKernelProgramOffsetHOSTKICK 100262e8     srvinitsgx:sgxinit.obj
 0002:0000f2ec       ui32uKernelProgramOffsetGETMISCINFO 100262ec     srvinitsgx:sgxinit.obj
 0002:0000f2f0       ui32uKernelProgramOffsetELB_PDSCONSTSIZE 100262f0     srvinitsgx:sgxinit.obj
 0002:0000f2f4       ui32uKernelProgramOffsetELB_PDSDEVADDR 100262f4     srvinitsgx:sgxinit.obj
 0002:0000f2f8       ui32uKernelProgramOffsetTA_ELB_PDSCONSTSIZE 100262f8     srvinitsgx:sgxinit.obj
 0002:0000f2fc       ui32uKernelProgramOffsetTA_ELB_PDSDEVADDR 100262fc     srvinitsgx:sgxinit.obj
 0002:0000f300       ui32uKernelProgramOffset3D_ELB_PDSCONSTSIZE 10026300     srvinitsgx:sgxinit.obj
 0002:0000f304       ui32uKernelProgramOffset3D_ELB_PDSDEVADDR 10026304     srvinitsgx:sgxinit.obj
 0002:0000f768       gpsResList                 10026768     srvkmcmn:resman.obj
 0002:0000f76c       gpsKernelHandleBase        1002676c     srvkmcmn:handle.obj
 0002:0000f7c8       gpsSysData                 100267c8     system:sysconfig.obj
 0002:0000f850       _exitflag                  10026850     corelib0:cexit.obj
 0002:0000f854       gui32EventStatusServicesByISR 10026854     srvkmsgx:sgxinit.obj
 0002:0000f86c       ui32uKernelProgramOffsetTA_TAHANDLER 1002686c     srvinitsgx:sgxinit.obj
 0002:0000f870       ui32uKernelProgramOffset3D_THREEDHANDLER 10026870     srvinitsgx:sgxinit.obj
 0002:0000f880       sEnvData                   10026880     <common>
 0002:0000f8b8       hBridgeMutex               100268b8     <common>
 0002:0000f8bc       gsSysSpecificData          100268bc     <common>
 0002:0000f8c0       gsSysData                  100268c0     <common>
 0002:0000f960       g_BridgeDispatchTable      10026960     <common>
 0002:0000fb18       __onexitend                10026b18     <common>
 0002:0000fb1c       __onexitbegin              10026b1c     <common>
 0002:0000fb20       _pRawDllMain               10026b20     <common>

 entry point at        0001:000105a8

 Static symbols

 0001:0000107c       FreeMappedClientMemInfo    1000207c f   pvr_bridge_k.obj
 0001:00001190       FreeUserModeMappingCallback 10002190 f   pvr_bridge_k.obj
 0001:000011fc       FreeSingleProcessUserModeMappingCallback 100021fc f   pvr_bridge_k.obj
 0001:00001260       RemapClientMemInfoFromUMAddr 10002260 f   pvr_bridge_k.obj
 0001:0000137c       RemapClientMemInfo         1000237c f   pvr_bridge_k.obj
 0001:00002390       OSTimerCallbackWrapper     10003390 f   osfunc_srvkm.obj
 0001:00004228       FreePerProcessData         10005228 f   srvkmcmn:perproc.obj
 0001:00004680       FreeResourceByPtr          10005680 f   srvkmcmn:resman.obj
 0001:000046f8       FreeResourceByCriteria     100056f8 f   srvkmcmn:resman.obj
 0001:00004fd0       CloseDCDeviceCallBack      10005fd0 f   srvkmcmn:deviceclass.obj
 0001:00005318       DestroyDCSwapChainCallBack 10006318 f   srvkmcmn:deviceclass.obj
 0001:00005be8       CloseBCDeviceCallBack      10006be8 f   srvkmcmn:deviceclass.obj
 0001:00005fb4       GetHandleStructure         10006fb4 f   srvkmcmn:handle.obj
 0001:00006004       FreeHandle                 10007004 f   srvkmcmn:handle.obj
 0001:000061a4       ReallocHandleArray         100071a4 f   srvkmcmn:handle.obj
 0001:00006270       IncreaseHandleArraySize    10007270 f   srvkmcmn:handle.obj
 0001:0000636c       AllocHandle                1000736c f   srvkmcmn:handle.obj
 0001:00006a10       PVRSRVHandleBatchCommitOrRelease 10007a10 f   srvkmcmn:handle.obj
 0001:00006b84       FreeHandleBase             10007b84 f   srvkmcmn:handle.obj
 0001:00006e54       PVRSRVDevicePrePowerStateKM 10007e54 f   srvkmcmn:power.obj
 0001:00006f00       PVRSRVDevicePostPowerStateKM 10007f00 f   srvkmcmn:power.obj
 0001:00007474       _RequestAllocFail          10008474 f   srvkmcmn:ra.obj
 0001:0000747c       _SegmentListInsert         1000847c f   srvkmcmn:ra.obj
 0001:00007520       _SegmentSplit              10008520 f   srvkmcmn:ra.obj
 0001:000075d4       _FreeListInsert            100085d4 f   srvkmcmn:ra.obj
 0001:0000761c       _InsertResource            1000861c f   srvkmcmn:ra.obj
 0001:000076d0       _InsertResourceSpan        100086d0 f   srvkmcmn:ra.obj
 0001:00007880       _FreeBT                    10008880 f   srvkmcmn:ra.obj
 0001:00007c4c       _AttemptAllocAligned       10008c4c f   srvkmcmn:ra.obj
 0001:000086a0       ZeroBuf                    100096a0 f   srvkmcmn:buffer_manager.obj
 0001:0000884c       BM_DestroyContextCallBack  1000984c f   srvkmcmn:buffer_manager.obj
 0001:00008bec       DevMemoryAlloc             10009bec f   srvkmcmn:buffer_manager.obj
 0001:00008d3c       BM_ImportMemory            10009d3c f   srvkmcmn:buffer_manager.obj
 0001:00008fcc       BM_FreeMemory              10009fcc f   srvkmcmn:buffer_manager.obj
 0001:00009120       AllocMemory                1000a120 f   srvkmcmn:buffer_manager.obj
 0001:00009310       WrapMemory                 1000a310 f   srvkmcmn:buffer_manager.obj
 0001:0000962c       FreeBuf                    1000a62c f   srvkmcmn:buffer_manager.obj
 0001:0000a8d0       _Resize                    1000b8d0 f   srvkmcmn:hash.obj
 0001:0000b098       AllocDeviceMem             1000c098 f   srvkmcmn:devicemem.obj
 0001:0000b1a8       FreeDeviceMem              1000c1a8 f   srvkmcmn:devicemem.obj
 0001:0000b334       FreeDeviceMemCallBack      1000c334 f   srvkmcmn:devicemem.obj
 0001:0000b568       UnwrapExtMemoryCallBack    1000c568 f   srvkmcmn:devicemem.obj
 0001:0000b928       UnmapDeviceMemoryCallBack  1000c928 f   srvkmcmn:devicemem.obj
 0001:0000bcc8       UnmapDeviceClassMemoryCallBack 1000ccc8 f   srvkmcmn:devicemem.obj
 0001:0000c8b4       PVRSRVEnumerateDevicesBW   1000d8b4 f   srvkmbridged:bridged_pvr_bridge.obj
 0001:0000c8d4       PVRSRVAcquireDeviceDataBW  1000d8d4 f   srvkmbridged:bridged_pvr_bridge.obj
 0001:0000c930       PVRSRVCreateDeviceMemContextBW 1000d930 f   srvkmbridged:bridged_pvr_bridge.obj
 0001:0000cabc       PVRSRVDestroyDeviceMemContextBW 1000dabc f   srvkmbridged:bridged_pvr_bridge.obj
 0001:0000cb58       PVRSRVGetDeviceMemHeapInfoBW 1000db58 f   srvkmbridged:bridged_pvr_bridge.obj
 0001:0000cc94       PVRSRVAllocDeviceMemBW     1000dc94 f   srvkmbridged:bridged_pvr_bridge.obj
 0001:0000ce50       PVRSRVFreeDeviceMemBW      1000de50 f   srvkmbridged:bridged_pvr_bridge.obj
 0001:0000cef0       PVRSRVExportDeviceMemBW    1000def0 f   srvkmbridged:bridged_pvr_bridge.obj
 0001:0000cfac       PVRSRVMapDeviceMemoryBW    1000dfac f   srvkmbridged:bridged_pvr_bridge.obj
 0001:0000d168       PVRSRVUnmapDeviceMemoryBW  1000e168 f   srvkmbridged:bridged_pvr_bridge.obj
 0001:0000d1d8       PVRSRVMapDeviceClassMemoryBW 1000e1d8 f   srvkmbridged:bridged_pvr_bridge.obj
 0001:0000d3a0       PVRSRVUnmapDeviceClassMemoryBW 1000e3a0 f   srvkmbridged:bridged_pvr_bridge.obj
 0001:0000d408       PVRSRVWrapExtMemoryBW      1000e408 f   srvkmbridged:bridged_pvr_bridge.obj
 0001:0000d628       PVRSRVUnwrapExtMemoryBW    1000e628 f   srvkmbridged:bridged_pvr_bridge.obj
 0001:0000d690       PVRSRVGetFreeDeviceMemBW   1000e690 f   srvkmbridged:bridged_pvr_bridge.obj
 0001:0000d6b8       PVRMMapOSMemHandleToMMapDataBW 1000e6b8 f   srvkmbridged:bridged_pvr_bridge.obj
 0001:0000d6c8       PVRMMapReleaseMMapDataBW   1000e6c8 f   srvkmbridged:bridged_pvr_bridge.obj
 0001:0000d6d8       PVRSRVGetMiscInfoBW        1000e6d8 f   srvkmbridged:bridged_pvr_bridge.obj
 0001:0000d814       PVRSRVConnectBW            1000e814 f   srvkmbridged:bridged_pvr_bridge.obj
 0001:0000d828       PVRSRVDisconnectBW         1000e828 f   srvkmbridged:bridged_pvr_bridge.obj
 0001:0000d838       PVRSRVEnumerateDCBW        1000e838 f   srvkmbridged:bridged_pvr_bridge.obj
 0001:0000d85c       PVRSRVOpenDCDeviceBW       1000e85c f   srvkmbridged:bridged_pvr_bridge.obj
 0001:0000d90c       PVRSRVCloseDCDeviceBW      1000e90c f   srvkmbridged:bridged_pvr_bridge.obj
 0001:0000d978       PVRSRVEnumDCFormatsBW      1000e978 f   srvkmbridged:bridged_pvr_bridge.obj
 0001:0000d9c4       PVRSRVEnumDCDimsBW         1000e9c4 f   srvkmbridged:bridged_pvr_bridge.obj
 0001:0000da18       PVRSRVGetDCSystemBufferBW  1000ea18 f   srvkmbridged:bridged_pvr_bridge.obj
 0001:0000dacc       PVRSRVGetDCInfoBW          1000eacc f   srvkmbridged:bridged_pvr_bridge.obj
 0001:0000db14       PVRSRVCreateDCSwapChainBW  1000eb14 f   srvkmbridged:bridged_pvr_bridge.obj
 0001:0000dbf4       PVRSRVDestroyDCSwapChainBW 1000ebf4 f   srvkmbridged:bridged_pvr_bridge.obj
 0001:0000dc5c       PVRSRVSetDCDstRectBW       1000ec5c f   srvkmbridged:bridged_pvr_bridge.obj
 0001:0000dcd0       PVRSRVSetDCSrcRectBW       1000ecd0 f   srvkmbridged:bridged_pvr_bridge.obj
 0001:0000dd44       PVRSRVSetDCDstColourKeyBW  1000ed44 f   srvkmbridged:bridged_pvr_bridge.obj
 0001:0000ddb8       PVRSRVSetDCSrcColourKeyBW  1000edb8 f   srvkmbridged:bridged_pvr_bridge.obj
 0001:0000de2c       PVRSRVGetDCBuffersBW       1000ee2c f   srvkmbridged:bridged_pvr_bridge.obj
 0001:0000df38       PVRSRVSwapToDCBufferBW     1000ef38 f   srvkmbridged:bridged_pvr_bridge.obj
 0001:0000dfc8       PVRSRVSwapToDCSystemBW     1000efc8 f   srvkmbridged:bridged_pvr_bridge.obj
 0001:0000e040       PVRSRVOpenBCDeviceBW       1000f040 f   srvkmbridged:bridged_pvr_bridge.obj
 0001:0000e0f0       PVRSRVCloseBCDeviceBW      1000f0f0 f   srvkmbridged:bridged_pvr_bridge.obj
 0001:0000e15c       PVRSRVGetBCInfoBW          1000f15c f   srvkmbridged:bridged_pvr_bridge.obj
 0001:0000e1a4       PVRSRVGetBCBufferBW        1000f1a4 f   srvkmbridged:bridged_pvr_bridge.obj
 0001:0000e25c       PVRSRVAllocSharedSysMemoryBW 1000f25c f   srvkmbridged:bridged_pvr_bridge.obj
 0001:0000e324       PVRSRVFreeSharedSysMemoryBW 1000f324 f   srvkmbridged:bridged_pvr_bridge.obj
 0001:0000e38c       PVRSRVMapMemInfoMemBW      1000f38c f   srvkmbridged:bridged_pvr_bridge.obj
 0001:0000e53c       PVRSRVModifySyncOpsBW      1000f53c f   srvkmbridged:bridged_pvr_bridge.obj
 0001:0000e60c       MMU_GetPDDevPAddrBW        1000f60c f   srvkmbridged:bridged_pvr_bridge.obj
 0001:0000e6a8       PVRSRVInitSrvConnectBW     1000f6a8 f   srvkmbridged:bridged_pvr_bridge.obj
 0001:0000e6fc       PVRSRVInitSrvDisconnectBW  1000f6fc f   srvkmbridged:bridged_pvr_bridge.obj
 0001:0000e774       PVRSRVEventObjectWaitBW    1000f774 f   srvkmbridged:bridged_pvr_bridge.obj
 0001:0000e7b8       PVRSRVEventObjectOpenBW    1000f7b8 f   srvkmbridged:bridged_pvr_bridge.obj
 0001:0000e864       PVRSRVEventObjectCloseBW   1000f864 f   srvkmbridged:bridged_pvr_bridge.obj
 0001:0000ecb8       SGXGetClientInfoBW         1000fcb8 f   srvkmbridged:bridged_sgx_bridge.obj
 0001:0000ed00       SGXReleaseClientInfoBW     1000fd00 f   srvkmbridged:bridged_sgx_bridge.obj
 0001:0000ed50       SGXGetInternalDevInfoBW    1000fd50 f   srvkmbridged:bridged_sgx_bridge.obj
 0001:0000edbc       SGXDoKickBW                1000fdbc f   srvkmbridged:bridged_sgx_bridge.obj
 0001:0000efec       SGXScheduleProcessQueuesBW 1000ffec f   srvkmbridged:bridged_sgx_bridge.obj
 0001:0000f030       SGXSubmitTransferBW        10010030 f   srvkmbridged:bridged_sgx_bridge.obj
 0001:0000f1a0       SGXGetMiscInfoBW           100101a0 f   srvkmbridged:bridged_sgx_bridge.obj
 0001:0000f258       SGXDevInitPart2BW          10010258 f   srvkmbridged:bridged_sgx_bridge.obj
 0001:0000f648       SGXRegisterHWRenderContextBW 10010648 f   srvkmbridged:bridged_sgx_bridge.obj
 0001:0000f6f0       SGXUnregisterHWRenderContextBW 100106f0 f   srvkmbridged:bridged_sgx_bridge.obj
 0001:0000f758       SGXRegisterHWTransferContextBW 10010758 f   srvkmbridged:bridged_sgx_bridge.obj
 0001:0000f800       SGXUnregisterHWTransferContextBW 10010800 f   srvkmbridged:bridged_sgx_bridge.obj
 0001:0000f868       SGXFlushHWRenderTargetBW   10010868 f   srvkmbridged:bridged_sgx_bridge.obj
 0001:0000f8ac       SGX2DQueryBlitsCompleteBW  100108ac f   srvkmbridged:bridged_sgx_bridge.obj
 0001:0000f924       SGXFindSharedPBDescBW      10010924 f   srvkmbridged:bridged_sgx_bridge.obj
 0001:0000fb34       SGXUnrefSharedPBDescBW     10010b34 f   srvkmbridged:bridged_sgx_bridge.obj
 0001:0000fb9c       SGXAddSharedPBDescBW       10010b9c f   srvkmbridged:bridged_sgx_bridge.obj
 0001:0000fe44       SGXGetInfoForSrvinitBW     10010e44 f   srvkmbridged:bridged_sgx_bridge.obj
 0001:000104ac       _DllMainCRTStartupHelper   100114ac f   corelib0:pegdmain.obj
 0001:000106ec       doexit                     100116ec f   corelib0:cexit.obj
 0001:00010928       SGXCommandComplete         10011928 f   srvkmsgx:sgxinit.obj
 0001:0001092c       InitDevInfo                1001192c f   srvkmsgx:sgxinit.obj
 0001:00010c28       DevInitSGXPart1            10011c28 f   srvkmsgx:sgxinit.obj
 0001:00010e64       DevDeInitSGX               10011e64 f   srvkmsgx:sgxinit.obj
 0001:00011208       SGXGetBuildInfoKM          10012208 f   srvkmsgx:sgxinit.obj
 0001:00011c08       SGXCleanupHWRenderContextCallback 10012c08 f   srvkmsgx:sgxutils.obj
 0001:00011c3c       SGXCleanupHWTransferContextCallback 10012c3c f   srvkmsgx:sgxutils.obj
 0001:000123e4       SGXCleanupSharedPBDescCallback 100133e4 f   srvkmsgx:pb.obj
 0001:000124c4       SGXCleanupSharedPBDescCreateLockCallback 100134c4 f   srvkmsgx:pb.obj
 0001:000128dc       SGXGetTimingInfo           100138dc f   srvkmsgx:sgxpower.obj
 0001:00012a28       SGXPrePowerState           10013a28 f   srvkmsgx:sgxpower.obj
 0001:00012b1c       SGXPostPowerState          10013b1c f   srvkmsgx:sgxpower.obj
 0001:00012d64       SGXResetInvalDC            10013d64 f   srvkmsgx:sgxreset.obj
 0001:0001305c       _DeferredFreePageTable     1001405c f   srvkmsgx:mmu.obj
 0001:000131fc       _DeferredAllocPagetables   100141fc f   srvkmsgx:mmu.obj
 0001:00013b1c       MMU_MapPage                10014b1c f   srvkmsgx:mmu.obj
 0001:00014000       ScriptWriteSGXReg          10015000 f   srvinitsgx:sgxinit.obj
 0001:00014048       LoaduKernelProgram         10015048 f   srvinitsgx:sgxinit.obj
 0001:000140ac       LoaduKernel                100150ac f   srvinitsgx:sgxinit.obj
 0001:00014928       SetupuKernel               10015928 f   srvinitsgx:sgxinit.obj
 0001:00014b90       SGXInitialisePart2         10015b90 f   srvinitsgx:sgxinit.obj
 0001:00014e14       SGXDeinitialise            10015e14 f   srvinitsgx:sgxinit.obj
 0001:00014efc       SGXMiscInit                10015efc f   srvinitsgx:sgxinit.obj
 0001:000151c4       FreeSharedSysMemCallBack   100161c4 f   srvkmcmn:mem.obj
